:0200000480007A
:100000006F000005732F2034930F80006308FF03F7
:10001000930F90006304FF03930FB0006300FF038E
:10002000130F000063040F0067000F00732F2034CC
:1000300063540F006F00400093E19153171F0000BD
:1000400023223FFC171F000023200FFC6FF01FFF2F
:100050009300000013010000930100001302000050
:100060009302000013030000930300001304000038
:100070009304000013050000930500001306000020
:100080009306000013070000930700001308000008
:10009000930800001309000093090000130A0000F0
:1000A000930A0000130B0000930B0000130C0000D8
:1000B000930C0000130D0000930D0000130E0000C0
:1000C000930E0000130F0000930F0000732540F102
:1000D0006310050097020000938202017390523072
:1000E000735044749702000093820201739052305F
:1000F00073500018970200009382420273905230AE
:100100009B021000939252039382F2FF7390023B82
:100110009302F0017390023A73504030970200004E
:1001200093824201739052307350203073503030BC
:100130009301000097020000938202ED7390523009
:10014000130510001315F501635C05000F00F00F97
:10015000930110009308D005130500007300000000
:1001600093020000638A020073905210B7B200003D
:100170009B829210739022307350003097020000DF
:100180009382420173901234732540F17300203042
:1001900093012000B7000080130100003BD720002E
:1001A000B70300806318776093013000B7000080C8
:1001B000130110003BD72000B7030040631C775E9B
:1001C00093014000B7000080130170003BD720006E
:1001D000B70300016310775E93015000B700008001
:1001E0001301E0003BD72000B70302006314775CE3
:1001F00093016000B70000809B8010001301F001A4
:100200003BD72000930310006316775A93017000C8
:100210009300F0FF130100003BD720009303F0FF91
:10022000631A7758930180009300F0FF13011000C8
:100230003BD72000B70300809B83F3FF631C7756F6
:10024000930190009300F0FF130170003BD7200052
:10025000B70300029B83F3FF631E77549301A00052
:100260009300F0FF1301E0003BD72000B703040028
:100270009B83F3FF631077549301B0009300F0FF6A
:100280001301F0013BD72000930310006314775251
:100290009301C000B72021219B80101213010000A0
:1002A0003BD72000B72321219B831312631477507F
:1002B0009301D000B72021219B8010121301100060
:1002C0003BD72000B79390109B8303096314774EAC
:1002D0009301E000B72021219B80101213017000D0
:1002E0003BD72000B74342009B8323246314774C01
:1002F0009301F000B72021219B8010121301E00030
:100300003BD72000B78300009B8343486314774AA0
:1003100093010001B72021219B8010121301F001ED
:100320003BD7200093030000631677489301100128
:10033000B72021219B801012130100FE3BD7200023
:10034000B72321219B831312631677469301200163
:10035000B72021219B801012130110FE3BD72000F3
:10036000B79390109B830309631677449301300180
:10037000B72021219B801012130170FE3BD7200073
:10038000B74342009B8323246316774293014001C5
:10039000B72021219B8010121301E0FE3BD72000E3
:1003A000B78300009B834348631677409301500155
:1003B000B72021219B8010121301F0FF3BD72000B2
:1003C000930300006318773E9301C002B720F1FF4A
:1003D0009B8050349390C00093808067130100008D
:1003E0003BD72000B75334129B8383676314773C59
:1003F0009301D002B720F1FF9B8050349390C0004E
:1004000093808067130140003BD72000B74323014E
:100410009B8373566310773A9301E002B72009007B
:100420009B8050349390C00093808067130100003C
:100430003BD72000B75334929B838367631C773686
:100440009301F002B72009009B8050349390C000C4
:1004500093808067130140003BD72000B7432309F6
:100460009B8373566318773493016001B700008053
:1004700013017000BBD02000B7030001639C7032F1
:1004800093017001B70000801301E0003BD1200010
:10049000B703020063107132930180019300700072
:1004A000BBD010009303000063967030930190015D
:1004B00013020000B7000080130170003BD720003A
:1004C000130307001302120093022000E31452FEEC
:1004D000B70300016310732E9301A0011302000003
:1004E000B70000801301E0003BD72000130000009C
:1004F000130307001302120093022000E31252FEBE
:10050000B70302006318732A9301B00113020000BD
:10051000B70000801301F0013BD72000130000005A
:1005200013000000130307001302120093022000BF
:10053000E31052FE93031000631E73269301C00163
:1005400013020000B7000080130170003BD72000A9
:100550001302120093022000E31652FEB7030001BB
:10056000631A77249301D00113020000B7000080C2
:100570001301E000130000003BD72000130212001B
:1005800093022000E31452FEB703020063147722A3
:100590009301E00113020000B70000801301F00195
:1005A00013000000130000003BD7200013021200CC
:1005B00093022000E31252FE93031000631C771E87
:1005C0009301F00113020000B70000801300000047
:1005D000130170003BD72000130212009302200089
:1005E000E31452FEB70300016316771C9301000267
:1005F00013020000B7000080130000001301E000A8
:10060000130000003BD720001302120093022000C9
:10061000E31252FEB7030200631E77189301100223
:1006200013020000B7000080130000001300000058
:100630001301F0013BD720001302120093022000A7
:10064000E31252FE93031000631677169301200203
:100650001302000013017000B70000803BD7200098
:100660001302120093022000E31652FEB7030001AA
:100670006312771493013002130200001301E000AB
:10068000B7000080130000003BD7200013021200C7
:1006900093022000E31452FEB7030200631C77109C
:1006A00093014002130200001301F001B700008023
:1006B00013000000130000003BD7200013021200BB
:1006C00093022000E31252FE930310006314770E8E
:1006D0009301500213020000130170001300000088
:1006E000B70000803BD720001302120093022000C5
:1006F000E31452FEB7030001631E770A9301600200
:10070000130200001301E00013000000B700008096
:10071000130000003BD720001302120093022000B8
:10072000E31252FEB70302006316770893017002CA
:10073000130200001301F001130000001300000079
:10074000B70000803BD72000130212009302200064
:10075000E31252FE93031000631E7704930180029C
:100760009300F0003B5110009303000063147104E8
:1007700093019002930000023BD10000930300021A
:10078000631A71029301A002BB50000093030000A2
:10079000639270029301B002930000403711000091
:1007A0001B0101803BD02000930300006314700004
:1007B000631030020F00F00F63800100939111006D
:1007C00093E111009308D005138501007300000028
:1007D0000F00F00F930110009308D00513050000DF
:1007E00073000000731000C0000000000000000053
:0C07F000000000000000000000000000FD
:1010000000000000000000000000000000000000E0
:1010100000000000000000000000000000000000D0
:1010200000000000000000000000000000000000C0
:1010300000000000000000000000000000000000B0
:081040000000000000000000A8
:040000058000000077
:00000001FF
